:1000000088C001C2A1C0A0C09FC09EC09DC09CC0AE
:100010009BC09AC099C098C097C096C095C094C024
:1000200093C092C091C004030904180372006100D8
:10003000700068006E00650074002E006E006500A0
:1000400074000A033100300030003000050109045B
:10005000A1010901A100850109300931150026FF20
:100060000075089502810205091901290815002566
:1000700001750195088102C0C005010904A10109AB
:1000800001A100850209300931150026FF0075081D
:10009000950281020509190129081500250175013C
:1000A00095088102C0C005010904A1010901A10050
:1000B000850309300931150026FF00750895028176
:1000C0000205091901290815002501750195088106
:1000D00002C0C005010904A1010901A100850409AC
:1000E000300931150026FF007508950281020509C7
:1000F0001901290815002501750195088102C0C064
:1001000012010101000000088B2803000401010214
:10011000030111241FBECFE5D4E0DEBFCDBF10E048
:10012000A0E6B0E0ECE8FEE002C005900D92AC3A2B
:10013000B107D9F711E0ACEAB0E001C01D92AB30D5
:10014000B107E1F711D3A0C65BCF85B7836085BF48
:100150008BB780648BBF83EC8093E10008950F938D
:100160001F93CF93DF939091F10019160CF0AFC05D
:100170002091EE008091ED008D3209F09EC08AE55D
:10018000809361009B3009F098C0CCE0D0E0C21BA6
:10019000D109CB50DF4F8881807609F080C0109262
:1001A000DF008981882359F41092E0008FED90E000
:1001B0009093F0008093EF0030E822E077C0853024
:1001C00021F48A818093F20068C0863009F04AC029
:1001D0008B81813009F441C0823019F4CE0176D28E
:1001E00060C0833069F58A81882349F486E290E013
:1001F0009093F0008093EF0030EC24E057C0813002
:1002000049F48AE290E09093F0008093EF0030ECA4
:1002100028E14CC0823049F483E690E09093F000EE
:100220008093EF0030E826E141C08330E9F582E4B5
:1002300090E09093F0008093EF0030EC2CE036C01B
:10024000813249F48FEB90E09093F0008093EF00BF
:1002500030EC29E02BC0823239F5CE0137D2282F7D
:1002600030EC24C0883019F484EF90E00AC0893063
:1002700021F48A818093F40010C08A3049F48FED14
:1002800090E09093F0008093EF0030E821E00EC002
:100290008B3019F483EC8093E10030E806C0CE0186
:1002A00043D2282F30E802C030EC20E08F81882331
:1002B00039F48E81821728F003C030E880E001C055
:1002C000822F3093AC00809360001092F1008091F7
:1002D000610084FF49C0809160008F3F09F444C0F1
:1002E000182F893008F018E0811B809360008091FE
:1002F000AC0080FD02C00BE401C003EC8F5F809373
:10030000AC002091EF003091F00086FD05C0D901CE
:10031000912FE7EDF0E011C0A7EDB0E080E090E0B4
:1003200006C0F901E80FF91FE491ED930196181743
:10033000C1F705C08D91819391509923D9F7F901A7
:10034000E10FF11DF093F000E093EF0087ED90E0F6
:10035000612F55D0183019F08FEF80936000009313
:10036000D6001C5F109361009AE080B3857031F471
:100370009150D9F71092F2001092EC00DF91CF91DA
:100380001F910F9108951F93DC01162F8091620039
:1003900084FF0AC08091E10098E889278093E100FA
:1003A000912FE2EEF0E007C08AE580936200F8CF7B
:1003B0008D91819391509923D9F782EE90E0612F2E
:1003C0001ED01C5F109362001F910895A82FB92FB3
:1003D0008FEF9FEF41E050EA615070F02D9138E0CF
:1003E000722F782796958795269570FF02C08427EF
:1003F00095273A95A9F7F0CF809590950895E6DF77
:100400008D939D930895CF93CFB7CF93809BFECFCD
:10041000809B09C0809B07C0809B05C0809B03C058
:10042000809B01C09EC0DF93C091EE00DD27CB50C2
:10043000DF4F809B02C0DF91EBCF2F930F931F9371
:1004400000B32FEF00FB20F94F933F9310B34FEF12
:10045000012700FB21F93BE031C04E7F012F10B393
:10046000216028C0102F4D7F2260000000B329C0FA
:100470004B7F2460012F000010B32BC010B3477FC7
:1004800028602AC04F7E00B320612CC04F7D10B37E
:1004900020622FC04F7B00B3206432C0422700B3DC
:1004A00049934FEF0000102710FB20F910B315708F
:1004B000A9F1297F91F2012700FB21F900B3237FE5
:1004C00089F23150F0F1102710FB22F910B3277E8A
:1004D00079F2012700FB23F92F7C81F200B310276A
:1004E00010FB24F92F7971F200C010B3012700FB33
:1004F00025F92F7359F200C000B3102710FB26F91D
:10050000223040F200C010B3012700FB27F924304D
:1005100028F64F77206810B30000F9CF3B50319593
:10052000333010E41ABFB8F0C31BD0400881033C3D
:1005300041F10B3431F11981412F1F772091EC00EB
:10054000121731F4093691F10D3279F0013E69F05C
:1005500022272093F3003F914F911F910F912F91EC
:10056000DF91CF91CFBFCF9118950093F3003F91CA
:100570004F911F910F912F91DF91CAB7C6FD46CFC2
:10058000F0CF0091F300002331F31091F10011231B
:10059000A1F53430A2F13093F1000093ED001091F9
:1005A000EE003BE0311B3093EE0029C00091F100DA
:1005B00001301CF50AE547FD09C03091610034FDAA
:1005C00020C000936100C6EDD0E01FC030916200F2
:1005D00034FD17C000936200C1EED0E016C00527BD
:1005E00010E002BB1FC0052722C0052727C0052732
:1005F0002CC0052710E002BB33C04AE503C042ED22
:1006000001C0432FC4E1D0E032E011B31560909AED
:1006100002B311BB5F9355E020E820FF052702BB22
:10062000279517951C3FD8F620FF0527279502BB75
:1006300017951C3FC0F620FF05272795179502BB8D
:100640001C3F98F620FF0527279517951C3F02BBF6
:1006500070F600C0499120FF052702BB279517952A
:100660001C3F38F620FF0527279502BB17951C3F36
:1006700038F520FF05272795179502BB1C3F10F57D
:1006800020FF0527279517951C3F02BBE8F4242F70
:100690003A9519F60A7F5F9102BB00C01091F200F3
:1006A000C651D04011F01093EC0010E41ABF016065
:1006B00011B31A7F402F4A7F02BB11BB42BB4BCF05
:1006C0000527D3CF0527D8CF0527DDCFFC018081B3
:1006D000807641F58181863029F583818230D1F0A1
:1006E000823269F08130F1F48091B1009091B200D2
:1006F0009093F0008093EF008091B3000895809173
:10070000AE009091AF009093F0008093EF00809145
:10071000B000089587E790E09093F0008093EF0099
:1007200082E2089580E00895DC0127EB30E0309309
:10073000F0002093EF008C918076803299F411962E
:100740008C911197813071F41092B400E091B50052
:10075000F091B6000784F089E02DC90112966C91E2
:100760000995089580E00895BF92CF92DF92EF92AD
:10077000FF920F931F93DF93CF93CDB7DEB72897E8
:100780000FB6F894DEBF0FBECDBFFE01319688E0F4
:10079000DF011D928A95E9F7B89A87B3897F87BBF5
:1007A00088B3866088BBC09880E395E70197F1F72E
:1007B00086B390E08670907095958795823009F4A5
:1007C000B0D08AD2FC019093B6008093B5008381AB
:1007D00094819093AF008093AE0081818093B000AC
:1007E00087819085009731F09093B2008093B1009B
:1007F000858107C080E091E09093B2008093B100C2
:1008000033D38093B3008091B0008093900014BAEA
:100810008FEF85BB88EF82BB85E081BB11BA8FE08B
:1008200085BD84EC83BDE091B500F091B6000184F4
:10083000F285E02D099589DCE091B500F091B600D4
:100840000384F485E02D0995789490E8B92E81E031
:10085000C82ED12CA89583DC08B607FEFBCFB8BE06
:10086000E091B500F091B6000384F485E02D099580
:10087000FF2400E010E012C00584F685E02D802FF3
:100880008F5F0995882341F0C601002E02C0880FB2
:10089000991F0A94E2F7F82A0F5F1F4FE091B50005
:1008A000F091B6008081992787FD90950817190768
:1008B0001CF3FF2079F200E010E0EF2CFF24E7FCAE
:1008C000F09422C0C701002E02C0959587950A9426
:1008D000E2F780FF17C08091620084FF13C0602F91
:1008E0006F5F0784F089E02D87EB90E00995682F12
:1008F00087EB90E048DD02C032DCA8958091620071
:1009000084FFFACF0F5F1F4FE091B500F091B60062
:100910008081992787FD9095081719070CF09ACFC9
:10092000D1CF1092AA0008958091C300882309F4C2
:100930004DC0AC9A80E38A95F1F7AC9860E070E026
:1009400020E030E098E1892F8A95F1F7AD98660FA5
:10095000770F9B9B61609A9B7160892F8A95F1F755
:10096000AD9A2F5F3F4F2830310569F740E050E0E6
:1009700020E030E098E1892F8A95F1F7AD98440F97
:10098000550F9B9B41609A9B5160892F8A95F1F787
:10099000AD9A2F5F3F4F2830310569F780E090E036
:1009A00038E1232F2A95F1F7AD98232F2A95F1F7F7
:1009B000AD9A019688309105A1F76093C6007093B7
:1009C000C7004093C8005093C90008958091C500A6
:1009D000882309F475C0AC9A80E3982F9A95F1F7B3
:1009E000AC988A95F1F7C59A88E18A95F1F720E0ED
:1009F00030E050E060E098E1AD98892F8A95F1F7FA
:100A0000550F660F9B9B51609A9B6160AD9A892F31
:100A10008A95F1F72F5F3F4F2830310569F75093E2
:100A2000C6006093C80020E030E098E1AD98892FBF
:100A30008A95F1F7569566959B9B50689A9B6068DE
:100A4000AD9A892F8A95F1F72F5F3F4F28303105F6
:100A500069F7C59888E18A95F1F720E030E090E0E9
:100A600040E078E1AD98872F8A95F1F7990F440F10
:100A70009B9B91609A9B4160AD9A872F8A95F1F775
:100A80002F5F3F4F2830310569F79093CA0040939C
:100A9000CC0020E030E078E1AD98872F8A95F1F71F
:100AA000969546959B9B90689A9B4068AD9A872F38
:100AB0008A95F1F72F5F3F4F2830310569F749C01C
:100AC000AC9A80E38A95F1F7AC9820E030E050E0F2
:100AD00060E090E040E078E1872F8A95F1F7AD98EB
:100AE000550F660F990F440F9B9B51609A9B616055
:100AF000999B9160989B4160872F8A95F1F7AD9AF9
:100B00002F5F3F4F2830310539F75093C60060936F
:100B1000C8009093CA004093CC0020E030E078E118
:100B2000872F8A95F1F7AD985695669596954695D7
:100B30009B9B50689A9B6068999B9068989B4068C3
:100B4000872F8A95F1F7AD9A2F5F3F4F28303105F7
:100B500039F78091AA00882321F18091C4005F3F7A
:100B600011F4816001C08E7F8093C4008091C40025
:100B70006F3F11F4826001C08D7F8093C40080912B
:100B8000C4009F3F11F4846001C08B7F8093C40038
:100B90008091C4004F3F11F4886001C0877F80932B
:100BA000C4008091C40080FD50E05093C70081FDD7
:100BB00060E06093C90082FD90E09093CB0083FDDC
:100BC00040E04093CD0008951F931FB7F894A49A76
:100BD000A59A84B3807F84BB85B38F6085BBAD9AB3
:100BE000AC98BD9AC59A1092C4009EDE8091AA006E
:100BF000882321F58091C7008F3F29F48091C4009C
:100C000081608093C4008091C9008F3F29F4809156
:100C1000C40082608093C4008091CB008F3F29F490
:100C20008091C40084608093C4008091CD008F3F88
:100C300029F48091C40088608093C400AC9A80E35A
:100C40008A95F1F7AC9880E090E030E040E058E120
:100C5000252F2A95F1F7AD989B9905C08331910511
:100C600019F441E001C03F5F252F2A95F1F7AD9AB5
:100C700001968831910561F7442329F0373119F441
:100C800081E08093C300C5989A9B10C0AC9A90E312
:100C9000892F8A95F1F79A9909C0AC98892F8A957E
:100CA000F1F79A9B03C081E08093C500C59A9A9B97
:100CB00010C0AC9A90E3892F8A95F1F79A9909C0F0
:100CC000AC98892F8A95F1F79A9B03C081E08093B5
:100CD000C5001FBF1F9108958CE490E090939D0084
:100CE00080939C0089E990E00895CF93DF93EC0115
:100CF000653010F080E094C08091C300E62FFF279C
:100D0000E7FDF095882359F1DF0111972097F9F05D
:100D10006883FD01EA53FF4F808180FD02C090E8A7
:100D200001C09FEF81FD90E09983FD01EA53FF4FE1
:100D3000808182FD02C090E801C09FEF83FD90E0BA
:100D40009A83FD01EA53FF4F8081807F8B83FD01F1
:100D5000EA53FF4F8081A253BF4F8C9360C0DF01E5
:100D60001197209709F44FC06883BD01660F771F64
:100D7000FB01EA53FF4F808180FD02C090E801C073
:100D80009FEF81FD90E09983FB01EA53FF4F808143
:100D900082FD02C090E801C09FEF83FD90E09A833E
:100DA0008091C40090E00A2E02C0959587950A9420
:100DB000E2F7FB01EA53FF4F80FF03C08081807F91
:100DC00021C06081462F50E09A012074307075E098
:100DD000359527957A95E1F7CA018072907033E0D6
:100DE000959587953A95E1F7282B661F6627661F2C
:100DF000262B4071507055954795242B8181829503
:100E0000807F822B8B83FD01EE0FFF1FDF01AA5332
:100E1000BF4F8D919C91E253FF4F9183808384E07B
:100E2000DF91CF91089581509091C300A82FB0E039
:100E3000992361F020E0FD01E253FF4FAA53BF4F19
:100E40009C918081981771F021E00CC0BD01660F64
:100E5000771FCB018A539F4F62537F4F42E050E090
:100E600006D0282F822F089582E190E00895FB019B
:100E7000DC0104C08D910190801921F44150504053
:0C0E8000C8F7881B990B0895F894FFCF69
:100E8C00FF5A5A140334006E00650073003400736B
:100E9C00006E006500730009022200010100803C15
:100EAC0009040000010300000009210101000122D6
:100EBC0000000705810308000A04B40000000000CC
:0C0ECC000000E405940413077506010003
:00000001FF
